:103CDF000ECF0EBB0EA70E920E7C0E650E4D0E3440
:103CEF000E190DFE0DE10DC40DA50D850D640D42D0
:103CFF000D1E0CFA0CD40CAE0C860C5D0C330C089C
:103D0F000BDC0BB00B820B540B250AF50AC40A937C
:103D1F000A610A2F09FD09CA09960963092F08FCD0
:103D2F0008C808950861082E07FB07C8079607649F
:103D3F000733070206D206A206730645061705EAE1
:103D4F0005BF059305690540051704F004C904A3D1
:103D5F00047E045A0437041503F403D303B4039603
:103D6F000378035B033F0324030A02F002D702BF69
:103D7F0002A80292027C02670253023F022C021A2F
:103D8F00020801F701E601D601C701B801A9019C9C
:103D9F00018E018101740168015D01510146013CF1
:103DAF0001320128011F0115010D010400FC00F46F
:103DBF0000EC00E500DE00D700D000CA00C300BD54
:103DCF0000B800B200AD00A700A2009E00990094B9
:103DDF000090008C008700840080007C00780075C4
:103DEF000072006E006B0068006500620060005D8D
:103DFF00005A0058005500530051004E004C004A25
:103E0F0000480046004400430041003F003E003C94
:103E1F00003A0039003700360035003300320031E8
:103E2F00002F002E002D002C002B002A0029002827
:103E3F000027002600250024002300010C010104A7
:103E4F0002011E030A9604013205030306006407EC
:103E5F00010108000009015A0E01010F00011200B3
:103E6F006413010114013C1501FA1664FA17FFFFE0
:103E7F001D00072000072400022701012F013C30FD
:103E8F00010132010335FFFF3603073CFFFF3DFF02
:103E9F00FF180002191E461A00021B00022D32C81D
:103EAF002E0001FAFAFA18000019FFFF1A00001B82
:0B3EBF0000002D32C82E0001FAFAFAB4
:10004800900786E0FEA3E0FF7457BE0010D39F40E0
:100058000C903E4912001EE493F599802F900014ED
:10006800E0D394044014900786E0FEA3E0FF903E9E
:100078004912001EE493F5998012900786E0FEA3CA
:10008800E0FF903E5E12001EE493F59990078612F9
:10009800000E900786E0FEA3E0FF746C6F4E7003BD
:1000A80075130022900072E0B40208740190007287
:1000B800F0D20D90013AE090002AF090013BE090D8
:1000C800002BF090013CE090002CF0A20AB34016FF
:1000D80090013AE0700C90013BE0700690013CE022
:1000E80060028002C20A90013AE0B4300F90013BEE
:1000F800E0B4470890013CE0643B60028004D20C05
:100108008002C20CE558B40102800302022E90005E
:1001180057E0F566900062E0F568900063E0F569E5
:10012800900074E0F56A90007AE0900029F0900061
:100138007CE0F56590007DE0F567900080E0F5646F
:10014800900081E0F563900090E0900041F090000D
:1001580091E0900042F0900092E0900043F090000F
:1001680093E0900044F0900094E0900045F09000F7
:1001780095E0900046F0900096E0900047F09000DF
:1001880097E0900048F0900099E0900033F09000DC
:100198009AE0900034F090009BE0900035F09000D9
:1001A8009CE0900036F0900079E0B4011790000AC6
:1001B800740FF0A374FFF090000CE4F0A3F0740245
:1001C800900079F0900079E0B4035990000CE0FEBB
:1001D800A3E0FF90000AE0FCA3E0FD120003741006
:1001E80012402A740812401CEF900026F0EF7006A7
:1001F80074FF900026F07400900079F090000BE0F6
:10020800900027F090000AE0900028F0900026E087
:10021800900789F0900027E090078AF0900028E086
:1002280090078BF0803F900081E07006755801754B
:100238006300A20AB3402E90013AE090002AF090A1
:10024800013BE090002BF090013CE090002CF090F6
:10025800002AE0700C90002BE0700690002CE06003
:10026800028002C20AE5667003756602E5687003DB
:100278007568027E887F4DE5668E048F05FF124003
:100288000C8C398D3AE56975F0FAA4FFAEF0E56893
:100298008E048F05FF12400C8C3D8D3E90004FE080
:1002A800F56090004DE0FE900069E0B506189000FA
:1002B8004CE0FE900068E0B5060C90004BE0FE9024
:1002C8000059E06E606F900069E07006900068E089
:1002D80060067400900059F0900069E0B40208903C
:1002E80000497401F08005900049E4F0900068E04E
:1002F800B4020890004A7401F0800590004AE4F0C6
:10030800900068E0600690004AE060028005756031
:10031800038003756004E559B55802D20D90006852
:10032800E090004CF0900069E090004DF09000598A
:10033800E090004BF0740190009EF0740190009FD3
:10034800F074009000A0F074009000A1F074009088
:1003580000A2F074009000A3F074009000A4F07460
:10036800019000A5F074019000A6F074009000A719
:10037800F074009000A8F074009000A9F074009048
:1003880000AAF074009000ABF074019000ACF07417
:10039800019000ADF074009000AEF074009000AFD2
:1003A800F074009000B0F074009000B1F074009008
:1003B80000B2F07401900362F07401900363F0746A
:1003C80000900364F07400900365F0740090036675
:1003D800F07400900367F07400900368F074009064
:1003E80003A2F074019003A3F074019003A4F074C5
:1003F800009003A5F074009003A6F074009003A782
:10040800F074009003A8F074009003E2F074009078
:1004180003E3F074019003E4F074009003E5F074D2
:10042800009003E6F074009003E7F074009003E88E
:10043800F07401900422F07400900423F074019089
:100448000424F07400900425F07400900426F074DD
:1004580000900427F07400900428F022E5B554F7C2
:10046800F5B5E5B554FDF5B5C2A2C2A1C292C20761
:10047800C297C2A0E5B554FBF5B5755104E5510422
:10048800F55290004FE0F560900025E4F0C209E5D0
:10049800B554FEF5B5C28E758D00758B00754C0090
:1004A800752600752500D28E22750A00750900AEE2
:1004B80009AF0A7457BE00039F500302056E903EB1
:1004C8004912001EE49390004E1240420FBF0001F3
:1004D8000EE0FC903E4912001EECFEE493FFEEC3D2
:1004E8009F5026AE09AF0A0FBF00010E903E491279
:1004F800001EAE09AF0AE493FC903E4912001EE4C8
:100508009390004E124042ECF0AE09AF0A903E497B
:1005180012001EE49390004E124042E0FC903E4BC5
:1005280012001EECFCE493FDECD39D4019903E4B69
:1005380012001EE493FC903E4912001EE4939000C2
:100548004E124042ECF0AE09AF0A74022FFF500180
:100558000E8E098F0A780A740126F6500418E436BC
:10056800F640030204B722750A00750900AE09AF08
:100578000A7415BE00039F500302063C903EA01269
:10058800001EE49390004E1240420FBF00010EE09F
:10059800FC903EA012001EECFEE493FFEEC39F50B9
:1005A80026AE09AF0A0FBF00010E903EA012001E32
:1005B800AE09AF0AE493FC903EA012001EE49390AB
:1005C800004E124042ECF0AE09AF0A903EA0120075
:1005D8001EE49390004E124042E0FC903EA21200AE
:1005E8001EECFCE493FDECD39D4019903EA2120052
:1005F8001EE493FC903EA012001EE49390004E125D
:100608004042ECF0AE09AF0A740F6F4E7006750ADF
:1006180015750900AE09AF0A74022FFF50010E8E3E
:10062800098F0A780A740126F6500418E436F64051
:100638000302057522750A00750900AE09AF0A7430
:1006480015BE00039F500302070A903EB512001E14
:10065800E49390004E1240420FBF00010EE0FC9060
:100668003EB512001EECFEE493FFEEC39F5026AE8B
:1006780009AF0A0FBF00010E903EB512001EAE0969
:10068800AF0AE493FC903EB512001EE49390004E2E
:10069800124042ECF0AE09AF0A903EB512001EE4DB
:1006A8009390004E124042E0FC903EB712001EECC0
:1006B800FCE493FDECD39D4019903EB712001EE474
:1006C80093FC903EB512001EE49390004E124042F7
:1006D800ECF0AE09AF0A740F6F4E7006750A157507
:1006E8000900AE09AF0A74022FFF50010E8E098F60
:1006F8000A780A740126F6500418E436F640030214
:10070800064322054D22054C22054EC2CF2290F801
:1007180000E4936406600280FE75840175A7007585
:10072800FF80900788E4F075C91075A70F75A1C7F9
:1007380075A70075D90075CEFF75A70F75F1FE7501
:10074800F2FF75F33775F47875A4BA75A5FF75A629
:100758000775AE0075AFFF75D48175D5FF75D6FFE7
:1007680075D7FFC296C295C2A0C20BC297E5B55411
:10077800BFF5B5E5B554DFF5B5E5B554EFF5B5E525
:10078800B5547FF5B5E5B554F7F5B5E5B554FDF5C0
:10079800B575A70075A20175A14775F80975BC0163
:1007A80075BE0475BD6C75BE0775BDA075BE0875B0
:1007B800BD0175BC0075BB1875BC2075BA0875E815
:1007C8008075D11375A70F75E10575E20075C740EF
:1007D800759700759780740A123FFC7597C0E59766
:1007E8005420700280F8758F0275A700D2AF7598F3
:1007F8000075A90C75A70F75AB4375ADFB75AC1EDD
:1008080075A700758911758E00758C00758A00D2E0
:10081800A9D28C758D00758B00D2ABD28E75CD00A8
:1008280075CC0075CA0075CB00D2ADC2CFD2CA75DF
:1008380091047592007593CD75EF0675D94075CF03
:1008480001900786E4F0A3F0751300751400C299AF
:10085800D20AC20E12046474C8F51875170012265D
:100868000E75A70FE5FB90001AF0E5FA90001BF053
:10087800E5F990001CF075A70090F800E493F508DE
:10088800122745122C7F900789E0900026F09007E8
:100898008AE0900027F090078BE0900028F09007FE
:1008A8008CE0900029F090078DE0F56690078EE0C7
:1008B800F56890078FE0F569900790E0F56A900772
:1008C80091E0F565900792E0F567900793E0F5648D
:1008D800900794E0F563900795E090002AF0900760
:1008E80096E090002BF0900797E090002CF090078E
:1008F80098E0900041F0900799E0900042F090074E
:100908009AE0900043F090079BE0900044F0900735
:100918009CE0900045F090079DE0900046F090071D
:100928009EE0900047F090079FE0900048F0900705
:10093800A0E0900033F09007A1E0900034F0900719
:10094800A2E0900035F09007A3E0900036F0740024
:10095800900082F090013AE0700C90013BE0700644
:1009680090013CE060028004C20A8002D20A90F83A
:1009780007E493900021F0900021E0440A900021C0
:10098800F0900021E054FE900021F07406900012CF
:10099800F07402900013F090F802E493900014F0C1
:1009A8007403900015F07403900016F0740690001C
:1009B80017F07405900018F0900014E0B404067461
:1009C80004900018F07405900019F090F804E4936E
:1009D80090001DF0740090001EF090F805E49390CC
:1009E800001FF090F806E493900020F074FF900048
:1009F80022F07447900125F0744D900126F0742080
:100A0800900127F07434900128F0744C900129F07B
:100A1800743690012AF0743090012BF074459001DF
:100A28002CF0742090012DF0742090012EF0742089
:100A380090012FF07434900130F07453900131F02C
:100A48007450900132F07444900133F090007AE0D1
:100A5800D394014006740090007AF07558017559D6
:100A680001740390004CF01200AC1204B190001411
:100A7800E0B4040512063D800312056F12263AE51C
:100A8800B554FEF5B5900025E4F0900786E4F0A390
:100A9800F0752400752300754800752A0075290033
:100AA800754900753200753100754A007554007536
:100AB8005500755A0075510475520175343C7533EB
:100AC80000757000756F007571CD7572CD75560023
:100AD80075570075430075440075450075460075E7
:100AE8005B00754700754200754100900006E4F010
:100AF800A3F0900008E4F0A3F0755E00755F009025
:100B0800000E74FDF0A374E8F0900023E4F0746420
:100B1800900024F0C200D201C202D203754D0075C4
:100B28006D00C294C293C287C290C291C20D7E0169
:100B38007F00900028E012402A900027E02FFF5005
:100B4800010E90000AEEF0A3EFF0900026E0700688
:100B580074FF900026F090000AE0FEA3E0FFEFD3B8
:100B680094FFEE940F400790000AE4F0A3F074009D
:100B7800900071F07400900079F07400900082F099
:100B8800740090008DF074009000B4F0E567700375
:100B9800756704743A90074EF074FD90074FF09013
:100BA80003D4E0900414F0D2B0D2B7D2A7D2A6D220
:100BB800B1D2A3C207A2B6B39204A2B3B39205D22C
:100BC8009CD2EC75CF01A298B34005C298122FE3CE
:100BD800E5136006A299B3B340028005C2991235A5
:100BE80053E51464016005E514B4040280D5E54DAD
:100BF800D39405400CE55AC394C85002055A754D64
:100C080000E571C394FA501A786F12003FAE6FAFC7
:100C180070EFD394E8EE9403400805717570007581
:100C28006F00C28E7E047F00E54C12402AE58D7568
:100C3800F004A4FDACF0EF2DFDEE3CFCE58B75F067
:100C48004084FF7E00ED2FFFEC3EFE8E258F26D2DE
:100C58008EA2B6300401B35003020D9EA2B6300432
:100C680001B35003020D9EA2B640670554A20E4080
:100C78000575FFA0D20EE5B54401F5B5900024E452
:100C8800F0E554D3956640487C887D4DAE25AF2667
:100C9800123ECA8E238F24E5482FFF50010E74019F
:100CA80012401C8E238F24852448755401C28E75EA
:100CB8008D00758B00754C00D28E7403BE00039FA7
:100CC80050069000257401F0E543B406037543000F
:100CD800D204A2B6B35003020D9EC20490006BE08A
:100CE8006018123694A200B34008E5B54408F5B57B
:100CF8008006E5B554F7F5B58002C20090006EE0B5
:100D080060181237E9A202B34008E5B54402F5B508
:100D18008006E5B554FDF5B58006E5B554FDF5B595
:100D2800A207B34004D2878002C287900059E060CE
:100D380004D2908002C29090004AE0B40104D29498
:100D48008002C294900049E0B40104D2938002C2A8
:100D580093A209B34004D2918002C291900018E096
:100D6800FE900014E0C39E4009900014E0D394085C
:100D7800400974FB900023F012046490001DE060A9
:100D88001590001DE0FE900017E06E600974FE905B
:100D98000023F0120464C2CA7E017F00E54E1240AF
:100DA8002AE5CD2FFF50010E8E278F28D2CAE56580
:100DB800B4014890000EE0FCA3E0FDEFC39DEE9C5B
:100DC8004039B208E52A45296013A208B34008E56E
:100DD800B54404F5B58006E5B554FBF5B590000EAD
:100DE800E0FEA3E0FF900010E0FCA3E0FDEF2DFD86
:100DF800EE3CFC90000EECF0A3EDF0A2B330050140
:100E0800B35003020EECA2B3300501B35003020E37
:100E1800ECA2B35003020EE50555A20E400575FF7E
:100E2800A0D20EE5B54401F5B5900024E4F0E555EF
:100E3800D395685003020EE37CEA7D60AE27AF28A5
:100E4800123ECA8E298F2AE56912402A74FF8E0441
:100E58008F05FF12400C8C298D2AE5492DFD500184
:100E68000C74018C068D0712401C8E298F2A852A46
:100E780049A209B34015746412402A900067E08EB5
:100E8800048F05FF12400C8C298D2A75550190009E
:100E98000EE0FEA3E0FFAC27AD2812000390000E81
:100EA800EEF0A3EFF0E567FF12400C740AFF124062
:100EB8000C90007BE08C068D0712402A74148E0477
:100EC8008F05FF12400C900010ECF0A3EDF0C2CAA1
:100ED80075CD0075CC00754E00D2CAD205A2B3B349
:100EE8004002C205900025E0B40107E556C3940608
:100EF80040030214FDE56D9025EDF8282873900055
:100F080059E0C39402400302105AE551D3940150AA
:100F18000302105AE55175F040A4FFAEF090031299
:100F280012001EE0C395455018E55175F040A4FF26
:100F3800AEF090031112001EE0F52E752D00021080
:100F48005AE55175F040A4FFAEF090031012001E50
:100F5800E0C395454003020FF6E55175F040A4FF44
:100F6800AEF090031112001EE55175F040A4FFAEDB
:100F7800F0E0FC90030F12001EECFEE0FFEEC39FB2
:100F8800FEE5518E0475F040A4FFAEF090031012F8
:100F9800001EE0F40425458C0088F0A4FFAEF0E5BF
:100FA800518F048E0575F040A4FFAEF09003121225
:100FB800001EE55175F040A4FFAEF0E0FA90031072
:100FC80012001EEAFEE0FFEEC39FFECDCCCD8E07D9
:100FD80012400CE55175F040A4FFAEF090030F12DB
:100FE800001EE02DFD50010C8C2D8D2E8064E551E6
:100FF80075F040A4FFAEF090030F12001EE5517586
:10100800F040A4FFAEF0E0FC90030E12001EECFED0
:10101800E0FFEEC39F8545F0A4FFAEF0E5518F04D5
:101028008E0575F040A4FFAEF090031012001EE08C
:10103800FECDCCCD8E0712400CE55175F040A4FFD3
:10104800AEF090030E12001EE02DFD50010C8C2D09
:101058008D2E756D010214FD900059E0C394024075
:101068000302120D90004FE0D3955150030211B6C0
:10107800E55175F040A4FFAEF090031812001EE091
:10108800C395455018E55175F040A4FFAEF09003A4
:101098001712001EE0F52C752B000211B6E55175EC
:1010A800F040A4FFAEF090031612001EE0C3954571
:1010B8004003021152E55175F040A4FFAEF09003D1
:1010C8001712001EE55175F040A4FFAEF0E0FC9049
:1010D800031512001EECFEE0FFEEC39FFEE5518EE5
:1010E8000475F040A4FFAEF090031612001EE0F461
:1010F8000425458C0088F0A4FFAEF0E5518F048EDE
:101108000575F040A4FFAEF090031812001EE551DB
:1011180075F040A4FFAEF0E0FA90031612001EEA44
:10112800FEE0FFEEC39FFECDCCCD8E0712400CE54E
:101138005175F040A4FFAEF090031512001EE02D8B
:10114800FD50010C8C2B8D2C8064E55175F040A46A
:10115800FFAEF090031512001EE55175F040A4FF94
:10116800AEF0E0FC90031412001EECFEE0FFEEC3AC
:101178009F8545F0A4FFAEF0E5518F048E0575F00C
:1011880040A4FFAEF090031612001EE0FECDCCCDB9
:101198008E0712400CE55175F040A4FFAEF09003A5
:1011A8001412001EE02DFD50010C8C2B8D2CE551E6
:1011B800B40122E560D39401401BE551C395565014
:1011C80014E545C39405500D90035FE0A829B800C5
:1011D80006952A40028003755102E551B5602290B8
:1011E800004FE0D395514019E55175F040A4FFAE8A
:1011F800F090031712001EE0A823B80006952440BB
:101208000280020560756D020214FD900059E0B479
:10121800022AE55175F040A4FFAEF09003171200C2
:101228001EE0F52C752B00E55175F040A4FFAEF0DB
:1012380090030E12001EE0F52E752D00900059E067
:10124800B4030F900051E0F52C752B00752E007536
:101258002D00756D030214FDE55175F040A4FFAE35
:10126800F090032012001EE0C3955A400302133485
:10127800900049E07036E551D394014029AE23AF80
:1012880024AC2DAD2EEDD39FEC9E401AE55175F0A0
:1012980040A4FFAEF090031E12001EE0A829B8007B
:1012A80005D3952A5002800215518034E551D39414
:1012B800024029AE23AF24AC2DAD2EEDD39FEC9E7A
:1012C800401AE55175F040A4FFAEF090031E1200DD
:1012D8001EE0A829B80005D3952A500280021551AE
:1012E800E551B55236E551C39560502FE551C39588
:1012F800565028AE23AF24AC2BAD2CEFD39DEE9CDB
:101308004019E55175F040A4FFAEF090031F12009C
:101318001EE0A829B80006952A400280020551C29D
:1013280092E55165526005C207755A00756D040251
:1013380014FDE55175F040A4FFAEF090031A1200B9
:101348001EE0B40117E55175F040A4FFAEF090031C
:101358002012001EE0240AC3955A400302140A759D
:101368003064752F00A207B3500B900060E024058D
:10137800C39545400302140AE55175F040A4FFAE39
:10138800F090031D12001EE0C395454064E55175B9
:10139800F040A4FFAEF090031C12001EE55175F05A
:1013A80040A4FFAEF0E0FC90031B12001EECFEE030
:1013B800FFEEC39F8545F0A4FFAEF0E5518F048E84
:1013C8000575F040A4FFAEF090031D12001EE0FE6C
:1013D800CDCCCD8E0712400CE55175F040A4FFAE80
:1013E800F090031B12001EE02DFD50010C8C2F8D78
:1013F80030AE23AF24AC2FAD30EFD39DEE9C40022E
:10140800D207756D050214FDE551B4010990005924
:10141800E0C3940240030214DD900358E0D39545DD
:1014280050030214DD900356E0C3954550409003E5
:1014380057E0FE900355E0F4042EFE900356E0F4C6
:101448000425458E0088F0A4FFAEF0900358E0FC18
:10145800900356E0F4042C8E048F05FF12400C9084
:101468000355E02DFD50010C8C2B8D2C802C900306
:1014780055E0FE900354E0F4042E8545F0A4FFAE39
:10148800F0900356E08E048F05FF12400C90035431
:10149800E02DFD50010C8C2B8D2CE551C39560502F
:1014A8002FE551C395565028AE23AF24AC2BAD2C55
:1014B800EFD39DEE9C4019E55175F040A4FFAEF0C6
:1014C80090031F12001EE0A829B80006952A4002C2
:1014D8008003755102900049E0B40106E5516401AA
:1014E80060028003755102E55165526005C20775B7
:0514F8005A00756D00B3
:1025ED00020F0602106002121302126002133A0269
:0225FD001410B8
:1014FD00900050E02402A823B80007D395244002A1
:10150D00C207900025E0B40109900059E0C394038F
:10151D004003021683900049E060030215D3E551A4
:10152D00D394014034E55175F040A4FFAEF0900323
:10153D001412001EE0A823B8001FD39524401AE50D
:10154D005175F040A4FFAEF090031F12001EE0A8ED
:10155D0029B80005D3952A500280021551E551D3C3
:10156D009401402FE55175F040A4FFAEF0900312A9
:10157D0012001EE0C39545501AE55175F040A4FFC9
:10158D00AEF090031E12001EE0A829B80005D395F9
:10159D002A500280021551E551D394014021E551A5
:1015AD00D39556401AE55175F040A4FFAEF0900367
:1015BD001E12001EE0A829B80005D3952A500280FE
:1015CD00021551021678E551D394024034E5517558
:1015DD00F040A4FFAEF090031412001EE0A823B853
:1015ED00001FD39524401AE55175F040A4FFAEF0CD
:1015FD0090031F12001EE0A829B80005D3952A50AC
:10160D000280021551E551D39402402FE55175F03A
:10161D0040A4FFAEF090031212001EE0C39545509A
:10162D001AE55175F040A4FFAEF090031E12001E96
:10163D00E0A829B80005D3952A500280021551E57E
:10164D0051D394024021E551D39556401AE5517579
:10165D00F040A4FFAEF090031E12001EE0A829B8C2
:10166D000005D3952A500280021551E5516552604F
:10167D0005C207755A00900060E0D395455009905A
:10168D000054E0C395455002C207900059E0700325
:10169D000218E6A2A5B34008A2A4B340030218CFD6
:1016AD00AE35AF367441D39F749C9E40057835128C
:1016BD00003FAE35AF36EFB48806EEB413028003AB
:1016CD000218ACA2A5500302176F900059E0B401A7
:1016DD000B90004FE0D3956040020560900059E0FB
:1016ED00B40253E55175F040A4FFAEF09003201203
:1016FD00001EE0C3955A503E90004FE0D3955140E7
:10170D0020E551C395565019E55175F040A4FFAE33
:10171D00F090031412001EE0A823B8000695244093
:10172D00028002055190004FE0F560E55165526071
:10173D0005C207755A00900059E0B4032590004F7B
:10174D00E0D395514007E551C395564002800205FF
:10175D005190004FE0F560E55165526005C2077587
:10176D005A00A2A450030218AC900059E0B4016EC7
:10177D00900049E07035E551D394014029E551754C
:10178D00F040A4FFAEF090031E12001EE0A829B891
:10179D00000FD3952A400A1551755A008551608066
:1017AD000385516080037560018033E551D3940248
:1017BD004029E55175F040A4FFAEF090031E1200D4
:1017CD001EE0A829B8000FD3952A400A1551755A65
:1017DD000085516080038551608003756002900023
:1017ED0059E0D3940150030218A0E55175F040A4BF
:1017FD00FFAEF090032012001EE0C3955A40030285
:10180D0018A0900049E07041E551D394014034E5B2
:10181D005175F040A4FFAEF090031112001EE0A828
:10182D0023B8001FD39524401AE55175F040A4FF4D
:10183D00AEF090031E12001EE0A829B80005D39546
:10184D002A500280021551803FE551D39402403455
:10185D00E55175F040A4FFAEF090031112001EE0AB
:10186D00A823B8001FD39524401AE55175F040A464
:10187D00FFAEF090031E12001EE0A829B80005D39C
:10188D00952A500280021551E55165526005C20737
:10189D00755A00E556B40704055E8003755E00E5D4
:1018AD0063B4010EAE35AF36EF64407005EE649C47
:1018BD006002800EA2A54003755801A2A4400375D5
:1018CD005802A2A5B3B35006A2A4B3B3400280063A
:1018DD007536007535000219D4A2A5B34008A2A42F
:1018ED00B340030219C0AE35AF367441D39F749C1B
:1018FD009E4005783512003FAE35AF36EFB4880601
:10190D00EEB4130280030219C0A2A5406F900068C7
:10191D00E0605A90004AE0B4010790004AE4F0807C
:10192D000690004A7401F090004AE070057560035E
:10193D00800375600490004AE0B40104D2948002E3
:10194D00C294E551B4041AE55175F040A4FFAEF010
:10195D0090031E12001EE0A829B80005D3952A5049
:10196D00028008755103C207755A00800375600423
:10197D00E556B40704055E8003755E00A2A44033EE
:10198D00900069E06021900049E0B40107900049A2
:10199D00E4F080069000497401F0900049E0B40134
:1019AD0004D2938002C293E556B40704055E80030A
:1019BD00755E00A2A5B3B35006A2A4B3B3400280D6
:1019CD0006753600753500E558655960069000823C
:1019DD00E06003021B5CC29C751400751300C2CA43
:1019ED00E5589025FFF82828738012122C7F800D62
:0D19FD00122D588008122E318003122F0A7F
:0F25FF000219F60219F80219FD021A02021A0750
:101A0A00900029E090007AF0E566900057F0E568CA
:101A1A00900062F0E569900063F0E56A900074F066
:101A2A00E56590007CF0E56790007DF0E564900044
:101A3A0080F0E563900081F090002AE090013AF08E
:101A4A0090002BE090013BF090002CE090013CF0DC
:101A5A00900041E0900090F0900042E0900091F0F8
:101A6A00900043E0900092F0900044E0900093F0E0
:101A7A00900045E0900094F0900046E0900095F0C8
:101A8A00900047E0900096F0900048E0900097F0B0
:101A9A00900033E0900099F0900034E090009AF0C2
:101AAA00900035E090009BF0900036E090009CF0AA
:101ABA007400900082F07447900125F0744D9001F3
:101ACA0026F07420900127F07434900128F0744CA9
:101ADA00900129F0743690012AF0743090012BF0AD
:101AEA00744590012CF0742090012DF0742090011F
:101AFA002EF0742090012FF07434900130F074535A
:101B0A00900131F07450900132F07444900133F036
:101B1A009003D4E0900414F0743A90074EF074FDE8
:101B2A0090074FF01200AC900004E4F0A3F090008C
:101B3A00067475F0A37430F09000087475F0A374FD
:101B4A0030F0855859D2CA754C00D29C741B90004B
:101B5A0023F0E556C394065005E551B55202806755
:101B6A00C207E55175F040A4FFAEF09003221200BF
:101B7A001EE030E003D38001C39296E55175F04030
:101B8A00A4FFAEF090032312001EE030E003D380DE
:101B9A0001C39295E55175F040A4FFAEF09003247D
:101BAA0012001EE030E003D38001C3920B8551522C
:101BBA00AE29AF2A7405BE00039F5007E545D394AA
:101BCA000550028002D292E556D394055003021CB6
:101BDA00DBC207E551D394014073E55175F040A487
:101BEA00FFAEF090031E12001EE0A829B80007D32A
:101BFA00952A40021551E5516552604EE55175F03E
:101C0A0040A4FFAEF090032212001EE030E003D39E
:101C1A008001C39296E55175F040A4FFAEF090039F
:101C2A002312001EE030E003D38001C39295E551F0
:101C3A0075F040A4FFAEF090032412001EE030E0DD
:101C4A0003D38001C3920B855152021CDBE556B4C3
:101C5A0006279000ACE030E003D38001C39296904F
:101C6A0000ADE030E003D38001C392959000AEE06E
:101C7A0030E003D38001C3920BE556B407279000E6
:101C8A00A5E030E003D38001C392969000A6E0302D
:101C9A00E003D38001C392959000A7E030E003D31C
:101CAA008001C3920BE556B4082790009EE030E00D
:101CBA0003D38001C3929690009FE030E003D38063
:101CCA0001C392959000A0E030E003D38001C39253
:101CDA000B900072E06058E54575F00284FF7E00C3
:101CEA0090014E12001EE0F55CE54775F00A84FF8C
:101CFA007E0090024E12001EE0F55DE55C255DD384
:101D0A009464400BE55C255DC39464F55C800375BF
:101D1A005C00E55C75F00284FF7E008F5CEFC39483
:101D2A00335007EF24CDF55C8003755CFF801CE51A
:101D3A004575F00284FF7E0090014E12001EE07588
:101D4A00F00284FF7E00EF24CDF55CE55CD394EBD2
:101D5A004003755CEBE595C3955C4004C2A2800222
:101D6A00D2A2E556D394054002C207A207400775DE
:101D7A0071CDC2978002D297E595C395714004C28E
:101D8A00A18002D2A1A20BB340057572FA80037535
:101D9A0072CDE595C395724004C2A08002D2A0E537
:101DAA0043C3940640030223ACA2EDB350030223BB
:101DBA00ACC2EDE5436003021F0E7E017F00E5BE63
:101DCA0012402AE5BD2FFF50010E900000EEF0A34D
:101DDA00EFF0900029E0B401177E0F7FFF9000001A
:101DEA00E0FCA3E0FD120003900000EEF0A3EFF088
:101DFA00900079E0B4025B900000E0FEA3E0FF905F
:101E0A00000AE0FCA3E0FDEDD39FEC9E400F90009A
:101E1A0000E0F8A3E090000AC8F0A3C8F090000020
:101E2A00E0FEA3E0FF90000CE0FCA3E0FDEFD39DF1
:101E3A00EE9C400F900000E0F8A3E090000CC8F080
:101E4A00A3C8F0900000E0FEA3E0FF740412401C57
:101E5A008F44900079E07060900000E0FEA3E0FFFC
:101E6A0090000AE0FCA3E0FDEFD39DEE9C400D122A
:101E7A000003900000EEF0A3EFF08007900000E46A
:101E8A00F0A3F0900000E0FEA3E0FF741012402AD5
:101E9A00900026E08E048F05FF12400C900000ECA3
:101EAA00F0A3EDF07400D39D74019C4008900001EA
:101EBA00E0F54480037544FFE54475F00AA4FFAEDB
:101ECA00F074198E048F05FF12400C8D45ED2532F2
:101EDA00FFAE3150010E740112401C8F4585453208
:101EEA00753100EFD394624003754562900072E049
:101EFA0064016006900066E0600280057543018017
:101F0A000375BB17E543B401028003021FFE7E017D
:101F1A007F00E5BE12402AE5BD2FFF50010E90005A
:101F2A0000EEF0A3EFF0900072E0B4017EE53445D4
:101F3A00336025AC33AD341DBDFF011C8F028E0307
:101F4A008C068D07903CDF12002EE493FE740193F9
:101F5A00FFEFC39AEE9B400280057833124054AEDD
:101F6A0033AF3474B3BE0025D39F4021900000E004
:101F7A00FCA3E0FD0FBF00010E903CDF12002EE42F
:101F8A0093FE740193FFEDC39FEC9E400280057897
:101F9A003312003FAE33AF34E56A12402A74648EBE
:101FAA00048F05FF12400C8D478033900066E06075
:101FBA002D900000E0FEA3E0FFEFD39400EE94081A
:101FCA00400F900066E0B40104C2098002D2098081
:101FDA000D900066E0B40104D2098002C2099000A3
:101FEA0072E064026006900066E0600575BB1680C8
:101FFA0003754302E543B4020280030220EC7E012A
:10200A007F00E5BE12402AE5BD2FFF50010E900069
:10201A0000EEF0A3EFF0900072E0B4027EE53445E2
:10202A00336025AC33AD341DBDFF011C8F028E0316
:10203A008C068D07903B7512002EE493FE74019373
:10204A00FFEFC39AEE9B400280057833124054AEEC
:10205A0033AF3474B3BE0025D39F4021900000E013
:10206A00FCA3E0FD0FBF00010E903B7512002EE4A9
:10207A0093FE740193FFEDC39FEC9E4002800578A6
:10208A003312003FAE33AF34E56A12402A74648ECD
:10209A00048F05FF12400C8D478033900066E06084
:1020AA002D900000E0FEA3E0FFEFD39400EE940829
:1020BA00400F900066E0B40104C2098002D2098090
:1020CA000D900066E0B40104D2098002C2099000B2
:1020DA0072E07003754700900066E07002C20975ED
:1020EA00BB1FE543B403457E017F00E5BE12402ACB
:1020FA00E5BD2FFF50010E900000EEF0A3EFF07443
:10210A000912402A74E68E048F05FF12400C8C4196
:10211A008D42E54A2DFD50010C74018C068D071283
:10212A00401C8E418F4285424A75BB19E543B4046F
:10213A000280030222947E017F00E5BE12402AE556
:10214A00BD2FFF50010E900000EEF0A3EFF07404D3
:10215A0012401C8F4BE564B40102800302222175F0
:10216A006B00756B00E56BD39407400302220EE502
:10217A006B900041124042E0D3954B501AE56B90A8
:10218A000041124042E0F404254BFEE56B90003713
:10219A00124042EEF08017E56B900041124042E097
:1021AA00C3954BFEE56B900037124042EEF0E56BAB
:1021BA00C394044009900084E0C3956B503BE56BDF
:1021CA006029E56B900037124042FEE0FFEE900076
:1021DA003FE0D39F4013E56B900037124042E090F6
:1021EA00003FF0E56B900040F0800E900037E090E1
:1021FA00003FF07400900040F0786B740126F640BE
:10220A000302216F900040E0F4042408F556E556D5
:10221A00D394054002C292E564D39401402FE54B62
:10222A00D3946E4004D20F8002C20F755605E5643E
:10223A00B40205A20FB340028003755607E564B4E1
:10224A000306A20FB3B340028003755607E557652C
:10225A00566008E55104F552855657E556B4070805
:10226A00E5B54480F5B58006E5B5547FF5B5E55684
:10227A0064066005E556B40808E5B54410F5B5806E
:10228A0006E5B554EFF5B575BB13E543B405028011
:10229A00030223A87E017F00E5BE12402AE5BD2F76
:1022AA00FF50010E900000EEF0A3EFF0740412400C
:1022BA001C8F46E563B4020280030223A5756B00F6
:1022CA00756B00E56BD39403400302235CE56B90C6
:1022DA000033124042E0D39546501AE56B90003322
:1022EA00124042E0F4042546FEE56B90002D1240B0
:1022FA0042EEF08017E56B900033124042E0C3953E
:10230A0046FEE56B90002D124042EEF0E56B602927
:10231A00E56B90002D124042FEE0FFEE900031E0A6
:10232A00D39F4013E56B90002D124042E09000319C
:10233A00F0E56B900032F0800E90002DE0900031B5
:10234A00F07400900032F0786B740126F6400302B4
:10235A0022CD900082E07043E52A45296036E5588F
:10236A00C39403500A900032E004C39403400280ED
:10237A0007900032E004F558E558D39402400A90D9
:10238A000032E004D3940250028007900032E00445
:10239A00F5588007900032E004F55875BB180543DC
:1023AA00D2ECE55ED3940450030224AD75CF01C28A
:1023BA00A2AE35AF367488D39F74139E4005A2A58A
:1023CA00B34014AE35AF367488D39F74139E40055C
:1023DA00A2A4B340028048783512003FAE35AF362A
:1023EA00EFB4883BEEB41337A2A5B3500990004F5F
:1023FA00E0D395515002800405518011A2A5B35033
:10240A000890004FE0655160028002D207A2A4B38F
:10241A005007E551D39401500280041551C207A216
:10242A00A5B3B35006A2A4B3B34002800675360022
:10243A00753500E5516552604EE55175F040A4FFCF
:10244A00AEF090032212001EE030E003D38001C3F5
:10245A009296E55175F040A4FFAEF0900323120066
:10246A001EE030E003D38001C39295E55175F04038
:10247A00A4FFAEF090032412001EE030E003D380E4
:10248A0001C3920B855152A20740057571CD800395
:10249A007571FFE595C395714004C2A18002D2A16E
:1024AA000223B6A20EB3500DAE25AF2674E8C39F21
:1024BA0074039E4002800575FFA0D20EAE25AF269A
:1024CA00EFD39420EE944E50030225C1120464C245
:1024DA008E758D00758B00754C00D28EC207757093
:1024EA0000756F007571CD75510475240075230050
:1024FA00755400755A00C287900059E06004D29062
:10250A008002C29090004AE0B40104D2948002C2D0
:10251A0094900049E0B40104D2938002C293A209C4
:10252A00B34004D2918002C29190006BE06018120D
:10253A003694A200B34008E5B54408F5B58006E52F
:10254A00B554F7F5B58002C20090006EE06018122B
:10255A0037E9A202B34008E5B54402F5B58006E5BD
:10256A00B554FDF5B58006E5B554FDF5B590000EF8
:10257A0074FDF0A374E8F0E543B4060375430090D4
:10258A000025E4F0752600752500758D00758B0011
:10259A00754C00900024E0C394035008900024E096
:1025AA0004F080067403900024F0900024E0B40341
:1025BA0006E5B554FEF5B5AE27AF28EFD39410EE75
:1025CA009427401CC2CA75CD0075CC0075280075C9
:1025DA002700D2CA754E00752A0075290075550064
:0325EA00020BCB16
:10399B00000001000132016401960196020002123F
:1039AB0002240200020003000340038003C0040052
:1039BB000440048004C00500060006000600060053
:1039CB00060006000600060000FF013101630195A9
:1039DB0001FF01FF0211022302FF02FF02FF033F5F
:1039EB00037F03BF03FF043F047F04BF04FF05FFF6
:1039FB0006FF06FF06FF06FF06FF06FF06FF06FF94
:103A0B000FAA0FA50F9F0F9A0F940F8D0F870F8083
:103A1B000F780F710F680F600F570F4E0F450F3B4D
:103A2B000F300F250F1A0F0E0F020EF50EE80EDBDF
:103A3B000ECC0EBE0EAE0E9F0E8E0E7D0E6C0E5A63
:103A4B000E470E340E200E0C0DF70DE20DCB0DB5FF
:103A5B000D9D0D850D6D0D540D3A0D200D050CE9C9
:103A6B000CCE0CB10C940C760C580C3A0C1B0BFBBB
:103A7B000BDB0BBB0B9A0B790B570B350B130AF1AB
:103A8B000ACE0AAB0A870A640A400A1C09F809D451
:103A9B0009B0098C09670943091F08FB08D608B24E
:103AAB00088E086A0846082307FF07DC07B9079644
:103ABB0007730751072F070D06EC06CA06AA0689DE
:103ACB0006690649062A060A05EC05CD05B00592DE
:103ADB0005750558053C0520050504EA04CF04B51A
:103AEB00049C04820469045104390422040B03F47A
:103AFB0003DE03C803B2039D038903750361034D02
:103B0B00033B03280316030402F202E102D102C0B5
:103B1B0002B002A0029102820273026502570249AF
:103B2B00023C022F02220216020901FD01F201E6FC
:103B3B0001DB01D001C601BB01B101A7019D0194BD
:103B4B00018B0182017901700168016001580150FC
:103B5B000148014101390132012B0125011E0118D8
:103B6B000111010B010500FF00FA0FA60FA00F9921
:103B7B000F920F8B0F840F7C0F740F6B0F620F580C
:103B8B000F4E0F430F380F2C0F1F0F120F050EF791
:103B9B000EE80ED80EC80EB70EA50E930E800E6C47
:103BAB000E580E420E2C0E150DFD0DE40DCB0DB166
:103BBB000D950D790D5D0D3F0D200D010CE10CC028
:103BCB000C9E0C7C0C590C350C100BEA0BC40B9E89
:103BDB000B760B4F0B260AFD0AD40AAA0A800A554C
:103BEB000A2A09FF09D409A8097C0950092508F9F3
:103BFB0008CD08A10875084A081E07F307C8079DDA
:103C0B0007730749072006F706CE06A6067E06575A
:103C1B000630060A05E405BF059B057705540532FA
:103C2B00051004EF04CE04AE048F04710453043565
:103C3B00041903FD03E203C703AD0394037B036382
:103C4B00034B0334031E030802F302DE02CA02B65F
:103C5B0002A30291027F026D025C024C023C022C19
:103C6B00021D020E020001F201E401D701CA01BEDE
:103C7B0001B101A6019A018F0185017A01700166DC
:103C8B00015D0153014A0141013901310129012132
:103C9B0001190112010B010400FD00F700F000EA0D
:103CAB0000E400DE00D900D300CE00C900C400BF81
:103CBB0000BA00B500B100AD00A800A400A0009CA4
:103CCB00009900950091008E008A00870084008186
:043CDB00007E007BEC
:10260E00751A00751900AE19AF1AAC17AD18EDC3D7
:10261E009FEC9E401674FF123FFC75CF01781A7422
:10262E000126F6500418E436F650DB22900786E4B5
:10263E00F0A3F0751000750F00751300751400C22D
:10264E0010D21122C2AF75D900758F0375B7A5755B
:10265E00B7F190F800E4F0758F0175B7A575B7F175
:10266E00E50890F800F075B7A575B7F190F801E49C
:10267E00F075B7A575B7F190079DE090F802F0756B
:10268E00B7A575B7F19007A1E090F803F075B7A55F
:10269E0075B7F190079EE090F804F075B7A575B781
:1026AE00F190079FE090F805F075B7A575B7F1901A
:1026BE0007A0E090F806F075B7A575B7F19007A2E0
:1026CE00E090F807F0758F0075D940D2AF229007D1
:1026DE0088E0B4AB61C2AF75D90075B62275F5222C
:1026EE00758F0375B7A575B7F1740090F600F07588
:1026FE008F01750A00750900AE09AF0A7413BE008A
:10270E00279F402475B7A575B7F190078912001E53
:10271E00E0FC90F60012001EECF0780A740126F62A
:10272E00500418E436F650D0758F0075F51175B655
:10273E002075D940D2AF22C2AF75D90075F522757A
:10274E000A00750900AE09AF0A7413BE00229F403D
:10275E001F90F60012001EE493FC90078912001ED3
:10276E00ECF0780A740126F6500418E436F650D5CB
:10277E0075F51175D940D2AF22900788E0B4AA0240
:10278E0080030228C4C2AF75D90075B62275F52232
:10279E00758F0375B7A575B7F1740090EE00F075DF
:1027AE00B7A575B7F1740090F000F075B7A575B7C1
:1027BE00F1740090F200F075B7A575B7F174009042
:1027CE00F400F0758F01750A00750900AE09AF0AA5
:1027DE0074FFC39F74019E402475B7A575B7F19021
:1027EE00004E12001EE0FC90EE0012001EECF0787F
:1027FE000A740126F6500418E436F650CF750A0016
:10280E00750900AE09AF0A74FFC39F74019E402480
:10281E0075B7A575B7F190024E12001EE0FC90F050
:10282E000012001EECF0780A740126F6500418E42B
:10283E0036F650CF750A00750900AE09AF0A74FF5F
:10284E00C39F74019E402475B7A575B7F190044ED1
:10285E0012001EE0FC90F20012001EECF0780A74DA
:10286E000126F6500418E436F650CF750A007509A5
:10287E0000AE09AF0A74FFC39F74019E402475B762
:10288E00A575B7F190064E12001EE0FC90F40012F2
:10289E00001EECF0780A740126F6500418E436F6A1
:1028AE0050CF758F0075F51175B62075D940D2AF22
:1028BE00743A90074EF022900788E0B4AA02800383
:1028CE00022A02C2AF75D90075B62275F522758F30
:1028DE000375B7A575B7F1740090E600F075B7A54E
:1028EE0075B7F1740090E800F075B7A575B7F1747F
:1028FE000090EA00F075B7A575B7F1740090EC0082
:10290E00F0758F01750A00750900AE09AF0A74FFE4
:10291E00C39F74019E402475B7A575B7F190004E04
:10292E0012001EE0FC90E60012001EECF0780A7415
:10293E000126F6500418E436F650CF750A007509D4
:10294E0000AE09AF0A74FFC39F74019E402475B791
:10295E00A575B7F190024E12001EE0FC90E8001231
:10296E00001EECF0780A740126F6500418E436F6D0
:10297E0050CF750A00750900AE09AF0A74FFC39FE8
:10298E0074019E402475B7A575B7F190044E1200E0
:10299E001EE0FC90EA0012001EECF0780A7401268C
:1029AE00F6500418E436F650CF750A00750900AEDD
:1029BE0009AF0A74FFC39F74019E402475B7A575B5
:1029CE00B7F190064E12001EE0FC90EC0012001EB5
:1029DE00ECF0780A740126F6500418E436F650CF5F
:1029EE00758F0075F51175B62075D940D2AF743A52
:1029FE0090074EF022900788E0B4AA028003022BC3
:102A0E0040C2AF75D90075B62275F522758F037564
:102A1E00B7A575B7F1740090DE00F075B7A575B760
:102A2E00F1740090E000F075B7A575B7F1740090E1
:102A3E00E200F075B7A575B7F1740090E400F0757B
:102A4E008F01750A00750900AE09AF0A74FFC39FA6
:102A5E0074019E402475B7A575B7F190004E120013
:102A6E001EE0FC90DE0012001EECF0780A740126C7
:102A7E00F6500418E436F650CF750A00750900AE0C
:102A8E0009AF0A74FFC39F74019E402475B7A575E4
:102A9E00B7F190024E12001EE0FC90E00012001EF4
:102AAE00ECF0780A740126F6500418E436F650CF8E
:102ABE00750A00750900AE09AF0A74FFC39F740151
:102ACE009E402475B7A575B7F190044E12001EE016
:102ADE00FC90E20012001EECF0780A740126F6500B
:102AEE000418E436F650CF750A00750900AE09AF2A
:102AFE000A74FFC39F74019E402475B7A575B7F184
:102B0E0090064E12001EE0FC90E40012001EECF047
:102B1E00780A740126F6500418E436F650CF758FF5
:102B2E000075F51175B62075D940D2AF743A90077D
:102B3E004EF022900788E0B4AA028003022C7EC2D7
:102B4E00AF75D90075B62275F522758F0375B7A5C9
:102B5E0075B7F1740090D600F075B7A575B7F1741E
:102B6E000090D800F075B7A575B7F1740090DA0033
:102B7E00F075B7A575B7F1740090DC00F0758F0194
:102B8E00750A00750900AE09AF0A74FFC39F740180
:102B9E009E402475B7A575B7F190004E12001EE049
:102BAE00FC90D60012001EECF0780A740126F65046
:102BBE000418E436F650CF750A00750900AE09AF59
:102BCE000A74FFC39F74019E402475B7A575B7F1B3
:102BDE0090024E12001EE0FC90D80012001EECF087
:102BEE00780A740126F6500418E436F650CF750AAA
:102BFE0000750900AE09AF0A74FFC39F74019E40B1
:102C0E002475B7A575B7F190044E12001EE0FC9026
:102C1E00DA0012001EECF0780A740126F650041841
:102C2E00E436F650CF750A00750900AE09AF0A7486
:102C3E00FFC39F74019E402475B7A575B7F190062A
:102C4E004E12001EE0FC90DC0012001EECF0780A22
:102C5E00740126F6500418E436F650CF758F0075C1
:102C6E00F51175B62075D940D2AF743A90074EF073
:102C7E0022C2AF75D90075F522750A00750900AE2E
:102C8E0009AF0A74FFC39F74019E401F90EE00129D
:102C9E00001EE493FC90004E12001EECF0780A74B5
:102CAE000126F6500418E436F650D4750A0075095C
:102CBE0000AE09AF0A74FFC39F74019E401F90F0CF
:102CCE000012001EE493FC90024E12001EECF078EF
:102CDE000A740126F6500418E436F650D4750A002C
:102CEE00750900AE09AF0A74FFC39F74019E401FA1
:102CFE0090F20012001EE493FC90044E12001EECA3
:102D0E00F0780A740126F6500418E436F650D4759D
:102D1E000A00750900AE09AF0A74FFC39F74019EC5
:102D2E00401F90F40012001EE493FC90064E120019
:102D3E001EECF0780A740126F6500418E436F650AC
:102D4E00D475F51175D940D2AF22C2AF75D90075C1
:102D5E00F522750A00750900AE09AF0A74FFC39F0C
:102D6E0074019E401F90E60012001EE493FC90003A
:102D7E004E12001EECF0780A740126F6500418E488
:102D8E0036F650D4750A00750900AE09AF0A74FF05
:102D9E00C39F74019E401F90E80012001EE493FC36
:102DAE0090024E12001EECF0780A740126F65004C2
:102DBE0018E436F650D4750A00750900AE09AF0A4C
:102DCE0074FFC39F74019E401F90EA0012001EE420
:102DDE0093FC90044E12001EECF0780A740126F655
:102DEE00500418E436F650D4750A00750900AE0981
:102DFE00AF0A74FFC39F74019E401F90EC00120037
:102E0E001EE493FC90064E12001EECF0780A74013C
:102E1E0026F6500418E436F650D475F51175D940DF
:102E2E00D2AF22C2AF75D90075F522750A007509A9
:102E3E0000AE09AF0A74FFC39F74019E401F90DE5F
:102E4E000012001EE493FC90004E12001EECF0786F
:102E5E000A740126F6500418E436F650D4750A00AA
:102E6E00750900AE09AF0A74FFC39F74019E401F1F
:102E7E0090E00012001EE493FC90024E12001EEC35
:102E8E00F0780A740126F6500418E436F650D4751C
:102E9E000A00750900AE09AF0A74FFC39F74019E44
:102EAE00401F90E20012001EE493FC90044E1200AC
:102EBE001EECF0780A740126F6500418E436F6502B
:102ECE00D4750A00750900AE09AF0A74FFC39F746A
:102EDE00019E401F90E40012001EE493FC90064EEB
:102EEE0012001EECF0780A740126F6500418E4362F
:102EFE00F650D475F51175D940D2AF22C2AF75D93F
:102F0E000075F522750A00750900AE09AF0A74FF47
:102F1E00C39F74019E401F90D60012001EE493FCC6
:102F2E0090004E12001EECF0780A740126F6500442
:102F3E0018E436F650D4750A00750900AE09AF0ACA
:102F4E0074FFC39F74019E401F90D80012001EE4B0
:102F5E0093FC90024E12001EECF0780A740126F6D5
:102F6E00500418E436F650D4750A00750900AE09FF
:102F7E00AF0A74FFC39F74019E401F90DA001200C7
:102F8E001EE493FC90044E12001EECF0780A7401BD
:102F9E0026F6500418E436F650D4750A007509006A
:102FAE00AE09AF0A74FFC39F74019E401F90DC00F0
:102FBE0012001EE493FC90064E12001EECF0780AEE
:102FCE00740126F6500418E436F650D475F51175D2
:102FDE00D940D2AF22E51464046006E59964FF601F
:102FEE00028031A2104004D2108027E514600874CC
:102FFE00E62514900023F0E513600874F025139075
:10300E000023F0E514B4010280FE75140075130060
:10301E00C2108002C210E51490393EF8282873754C
:10302E001400E599B4FF03751301E599B4FE037519
:10303E001302E599B4FD03751303E599B4FC03750A
:10304E001304E599B4FA03751305E599B4FB0675F7
:10305E001401120464E599B4F9067514041204649B
:10306E00E599D394E54007E599C394F040028016A4
:10307E008599157514027E017F00E515C394E6123D
:10308E00402A8E0D8F0E900786E4F0A3F0E599D3BB
:10309E0094C44007E599C394E640028028859915AB
:1030AE0075140374E5C39515F50E750D00AE0DAFD1
:1030BE000E90399B12002EE493F8740193900786BC
:1030CE00C8F0A3C8F0D299023552900786E0FEA34D
:1030DE00E0FFEFC39400EE94054009EFD394FFEEAA
:1030EE0094064013900786E0FEA3E0FF90004E1278
:1030FE00001EE599F0800385996C90078612000EEC
:10310E00900786E0FEA3E0FFEFB40106EEB40702DF
:10311E00800302336290074EE0B43C028003023318
:10312E0062A20AB35005A20CB34003023255C29CF0
:10313E0090007AE090078CF0900057E090078DF0A9
:10314E00900062E090078EF0900063E090078FF0A1
:10315E00900074E0900790F090007CE0900791F062
:10316E0090007DE0900792F0900080E0900793F041
:10317E00900081E0900794F090013AE0900795F06E
:10318E0090013BE0900796F090013CE0900797F09D
:10319E00900090E0900798F0900091E0900799F0E1
:1031AE00900092E090079AF0900093E090079BF0C9
:1031BE00900094E090079CF0900095E090079DF0B1
:1031CE00900096E090079EF0900097E090079FF099
:1031DE00900099E09007A0F090009AE09007A1F07F
:1031EE0090009BE09007A2F090009CE09007A3F067
:1031FE007400900082F01200AC74AB900788F0124D
:0A320E0026DC74AA900788F0E5584A
:06393E0002302D0230D81A
:1032180090395FF82828738012122787800D1228AA
:0B322800C58008122A038003122B410E
:0F395F0002321F02322102322602322B02323094
:10323300900788E4F090013AE0700C90013BE07055
:103243000690013CE060028004C20A8002D20A02B6
:103253003357C29C900078E0900789F090005EE0BD
:1032630090078AF090005FE090078BF090007AE07F
:1032730090078CF0900057E090078DF0900062E08B
:1032830090078EF0900063E090078FF0900074E059
:10329300900790F090007CE0900791F090007DE023
:1032A300900792F0900080E0900793F0900081E007
:1032B300900794F090013AE0900795F090013BE07D
:1032C300900796F090013CE0900797F0900090E013
:1032D300900798F0900091E0900799F0900092E0A9
:1032E30090079AF0900093E090079BF0900094E091
:1032F30090079CF0900095E090079DF0900096E079
:1033030090079EF0900097E090079FF0900099E05F
:103313009007A0F090009AE09007A1F090009BE046
:103323009007A2F090009CE09007A3F07400900037
:1033330082F074AB900788F01226DC74AA90078899
:10334300F01227871228C5122A03122B41D29C752B
:1033530099FB80FED29C7514007513007599FB02CE
:103363003552900786E0FEA3E0FFEF4E7006859985
:1033730010750F00900786E0FEA3E0FF74016F4E07
:10338300701BAC0FAD10AA0DAB0EED2BFBEC3AFA94
:103393008A068B0790004E12001EE599F09007866F
:1033A30012000E900786E0FEA3E0FF74026F4E70DA
:1033B3000C1200AC85159975140075130002355273
:1033C300900786E0FEA3E0FF90004E12001EE599F1
:1033D300F090078612000E900786E0FEA3E0FFAC94
:1033E3000DAD0E8F028E038C068D079039D312001C
:1033F3002EE493F9740193FEEAD39EEB9940098579
:103403001599751400751300023552900786E0FE76
:10341300A3E0FF90004E12001EE599F0900786127C
:10342300000E900786E0FEA3E0FFEFB40006EEB4C3
:103433000102800302355290001CE0D394C7400B75
:1034430090001CE0C394C8F516801A90001CE0D3CA
:103453009463400B90001CE0C39464F516800690BF
:10346300001CE0F516E51675F002A4FFAEF08F6BB5
:10347300EF90004E124042EFFCE0FDEC9000511241
:103483004042EDFCE0FDEC2DB5160280030235440D
:103493000FEF90004E124042E56BFFE0FCEF90000F
:1034A30052124042ECFFE0FCEFC39CB516028003CE
:1034B300023544E56B900050124042E56BFFE0FC9F
:1034C300EF900053124042ECFFE0FCEF2CB5167175
:1034D300E56B900054124042E0C3951690079DF0AF
:1034E300E56B900055124042E0C3951690079EF09D
:1034F300E56B900058124042E0C3951690079FF089
:10350300E56B900059124042E0C395169007A0F076
:10351300E56B90005A124042E0C395169007A1F064
:10352300E56B90005B124042E0C395169007A2F052
:103533001226527599F975186475170012260E80B4
:0F354300FE7599FF75186475170012260E80FE2D
:093944000233650233C302340EA4
:1035520022E51390394DF828287302369390078696
:10356200E0FEA3E0FF90001212001EE0F599900722
:103572008612000E900786E0FEA3E0FF74116F4EE4
:103582007003751300023693856299023693900791
:1035920086E0FEA3E0FF90004E12001EE0F599EFD8
:1035A200B40107EEB4070375130090078612000EEC
:0735B200023693900787E049
:0F394D0002355C02355F02358A0235900235B5CE
:1035B90090396EF8282873852499023688852A99C6
:1035C9000236888544990236888547990236888566
:1035D900519902368885609902368885569902364E
:1035E90088855899023688756E00900069E07006E2
:1035F900900068E060028016A2A44006E56E4404CB
:10360900F56EA2A54006E56E4402F56E801A90009B
:103619004AE0B40106E56E4410F56E900049E0B445
:103629000106E56E4420F56EA207B34006E56E4437
:1036390001F56EA209B34006E56E4408F56E856E84
:1036490099803CA211B340077599FAC2118017A25B
:103659000DB3400575990F800B900023E0F5999003
:103669000023E4F0C20D80178542998012854B9999
:0F367900800D85469980087599FC8003751300B4
:10396E000235C00235C60235CC0235D20235D80238
:10397E0035DE0235E40235EA0235F002364C023607
:0D398E007102367602367B023680023685E5
:0B36880090078612000E80031200481D
:03395C00023690A0
:103693002290006BE0B4010385241190006BE0B429
:1036A3000203852A1190006BE0B403038544119053
:1036B300006BE0B4040385471190006BE0B405038D
:1036C30085511190006BE0B4060385561190006B91
:1036D300E0B4070385581190006CE0FE90006DE0A4
:1036E300C39E500302376A90006BE0D39404402CCE
:1036F30090006CE0D39511500990006DE0C39511D3
:1037030050028002D20090006CE0D39511500990D2
:10371300006DE0C395115002C200804990006BE038
:10372300B4041890006DE0C395115002D2009000CC
:103733006CE0D395114002C200802A90006CE0C374
:103743009511500990006DE0D3951150028002D27B
:103753000090006CE0D39511500990006DE0C39583
:10376300115002C200807E90006BE0D39404402C81
:1037730090006CE0C39511400990006DE0D3951162
:1037830040028002C20090006CE0C3951140099092
:10379300006DE0D395114002D200804990006BE0A8
:1037A300B4041890006CE0C395115002C20090005D
:1037B3006DE0D395114002D200802A90006CE0C3E3
:1037C3009511400990006DE0D395114002D200900D
:1037D300006CE0D39511400990006DE0C395114052
:1037E300028002C2002290006EE0B401038524111E
:1037F30090006EE0B40203852A1190006EE0B403DA
:103803000385441190006EE0B404038547119000D2
:103813006EE0B4050385511190006EE0B406038594
:10382300561190006EE0B4070385581190006FE0C5
:10383300FE900070E0C39E50030238BF90006EE01C
:10384300D39404402C90006FE0D39511500990005D
:1038530070E0C3951150028002D20290006FE0D352
:1038630095115009900070E0C395115002C2028077
:103873004990006EE0B40418900070E0C3951150B5
:1038830002D20290006FE0D395114002C202802A57
:1038930090006FE0C395115009900070E0D395112B
:1038A30050028002D20290006FE0D395115009902C
:1038B3000070E0C395115002C202807E90006EE05A
:1038C300D39404402C90006FE0C3951140099000FD
:1038D30070E0D3951140028002C20290006FE0C3F2
:1038E30095114009900070E0D395114002D20280F7
:1038F3004990006EE0B4041890006FE0C395115036
:1039030002C202900070E0D395114002D202802AD5
:1039130090006FE0C395114009900070E0D39511BA
:103923004002D20290006FE0D395114009900070DD
:0B393300E0C3951140028002C2022296
:094042002582F58250020583225B
:10002E00EF2F500205832582F582E5833E2EF58360
:01003E00229F
:08000300C3EF9DFFEE9CFE22FD
:08003F000806B60002180622B3
:0D000E00A3E004F07006124038E004F02278
:084054000816B6FF021816223F
:0E401C00048007C3CE13CECF13CFD5E0F6221B
:103ECA00BC000FBE0008ED8FF084FFADF022E4FEC7
:103EDA00FF22BE000DEF60FE54F0606F20E7030280
:103EEA003F80EAC0E0EBC0E078017A0075F001EEAD
:103EFA0020E710EF25E0FFEE33FE0AC5F023C5F0F8
:103F0A0030E7F0EA5407F9096A7A007B0060010891
:103F1A00C3EC9E40167004ED9F4010ED9FFDEC9E91
:103F2A00FCE5F0CA4ACA03F5F08005E5F003F5F0AE
:103F3A00C3EE13FEEF13FFD9D77908CACBCAD8D07C
:103F4A00EAFEEBFFD0E0FBD0E0FA22EC8FF084FC33
:103F5A00ED54F045F0C48FF084FEEDC454F045F002
:103F6A00C48FF084FDEEC4FE54F02DFFEE540F3CD6
:103F7A00FEADF07C0022790078008FF0EC7E0820FC
:103F8A00E70DC3CD33CD33C933C9C833C8DEF08496
:103F9A0049F9E5F08FF0BE00E6FD7C00E9FFE8FE96
:013FAA0022F4
:0E402A00F88FF0A4FFE5F0CE88F0A42EFE2261
:103FFC00600D782B024006007830D8FED5E0F82210
:10400C00EEC0E07E00123ECAEFFDEEFCD0E0FE22D8
:03000B00023FAB06
:03001B00023FC6DB
:03002B00023FE1B0
:0300000002404B70
:09404B0075817375D0000207169F
:0B001E00E5822FF582E5833EF583228A
:0A4038000582D5820215831582224D
:103FAB00C0E0C0F0C083C082C0D075D00012070B38
:103FBB00D0D0D082D083D0F0D0E032C0E0C0F0C0FF
:103FCB0083C082C0D075D00012070ED0D0D082D063
:103FDB0083D0F0D0E032C0E0C0F0C083C082C0D04C
:103FEB0075D000120711D0D0D082D083D0F0D0E0A2
:013FFB003293
:00000001FF
